:020000040000FA
:10000000F86A7D0EF76EC00EF66EA68EA69CA684CC
:10001000A688F29E550EA76EAA0EA76EA6820000B5
:10002000F28E010EF56E0D00EF0EF56E0D00300E26
:10003000F56E0D00F00EF56EF56A0D000D000D0069
:100040000C00A68EA69CA684A698F29E550EA76EBE
:10005000AA0EA76EA6820000F28EA6948E0EC16E26
:10006000E10E926E100E806E8082FFD701EF30F0AD
:10600000FFD7E0CF0AF50501F2AE03D0F29E128F62
:1060100001D0129FE8CF00F5D8CF01F5EACF02F505
:10602000E9CF03F5E2CF04F5E1CF05F5DACF06F5C8
:10603000D9CF07F5FBCF08F5FACF09F5F8CF0BF567
:10604000F7CF0CF5F6CF0DF5D5AE03D0D59E128166
:1060500001D01291CDA003D0CD90128301D0129324
:10606000CAA403D0CA94128501D01295B1A003D05E
:10607000B190128701D01297D49CBDEC30F059B585
:1060800001D0396BC4EC30F05851130B130A20E0E7
:1060900059B506D0596BCBEC36F06EEC35F001D02B
:1060A0005995126B0E6B0F6B106B116B58B310D0B0
:1060B000700EF76E9C0EF66E0BEC31F0700EF76EF4
:1060C000C00EF66E0BEC31F016EC31F09DEC31F0B9
:1060D00058AB24D0D4AA05D010C50EF511C50FF5C4
:1060E0001DD058AF12D080EC31F039B901D03983CE
:1060F000FECF10F5FDCF11F5710EF76E140EF66E92
:106100000BEC31F09DEC31F009D0D488B8500E6F13
:10611000B7500F6FD498D8900F370E37FECF10F5C9
:10612000FDCF11F558AB1AD0589B58AF0AD0D4BA4E
:1061300008D09EAA06D0710EF76E140EF66E0BEC08
:1061400031F058AD09D0589DD8EC36F0710EF76E8D
:10615000140EF66E0BEC31F01FEC37F0710EF76E8B
:10616000140EF66E0BEC31F0598147EC32F0599178
:10617000FCEC32F09DEC31F0F1D71F0EAF6EAC8429
:10618000AC8AAB88AB8E1200FCAC07D0FC9C740EC2
:10619000F76E5A0EF66E0BEC31F0FCAE07D0FC9E9B
:1061A000740EF76E480EF66E0BEC31F0D0501F0BEC
:1061B0001F0A0DE158AB0AD058AF07D0D4BA05D0AA
:1061C000A9EC32F09EBA01D0D09201D0D092D0B2D8
:1061D00006D0DD0E586F596BD082D08001D0588325
:1061E000D0B009D05891D080740EF76E2C0EF66E98
:1061F0000BEC31F001D05881D0B80BD05899D08831
:1062000059B506D0730EF76EE20EF66E0BEC31F058
:1062100001D0588912000800F55004D80B00F55041
:10622000FCE112009EA8FED7AD6E120080EC31F0AA
:1062300039B947D09EAA03D0AE509EBAFDD7020E00
:10624000136F1353D8B431D0730EF76E0A0EF66E77
:106250000BEC31F0730EF76E2E0EF66E0BEC31F088
:106260005B0E12EC31F0200E12EC31F0132FFBD745
:106270005D0E12EC31F0030E136F080E12EC31F0CC
:10628000132FFBD7020E136FABA202D0AB98AB88D3
:106290009EBA15D0640E146FA9EC32F01407FCE11D
:1062A000230E12EC31F0132FEFD7B9EC32F0710E50
:1062B000F76E140EF66E0BEC31F0398102D0B9ECAA
:1062C00032F012003989000EF76E000EF66E030EE2
:1062D000156F0900F55207E00900F550EF0801E1DC
:1062E00039990DD00AD00900F550EF0803E139992A
:1062F00006D003D0F55001E002D01507EAE1120004
:106300003989F76AF66A600E616F000E626F0900E4
:10631000F550FF0A01E009D0620701E2610762530C
:1063200003E1615301E101D0F2D7615304E162530B
:1063300001E0399901D03999120039AD09D0C9EC81
:1063400033F0710EF76EF20EF66E0BEC31F01DD0DD
:1063500039AF09D0C9EC33F0720EF76E100EF66E3D
:106360000BEC31F012D039A907D0720EF76E380E4F
:10637000F66E0BEC31F009D039A303D0C7EC31F045
:1063800004D039A102D003EC32F0396B12000600C0
:1063900006005851130B130A07E0FC2A000EFF6E8B
:1063A000000EFE6E000EFD6E588BD48AD48C12A1A6
:1063B00001D0D58E12A301D0CD8012A501D0CA8400
:1063C00012A701D0B18012AF01D0F28E0BC5F8FF39
:1063D0000CC5F7FF0DC5F6FF0AC5E0FF09C5FAFFBA
:1063E00008C5FBFF02C5EAFF03C5E9FF04C5E2FFDC
:1063F00005C5E1FF06C5DAFF07C5D9FF01C5D8FF0E
:1064000000C5E8FFE1000600060058AF06D0710E97
:10641000F76ECC0EF66E0BEC31F05851130B130ADD
:1064200007E0FC2A000EFF6E000EFE6E000EFD6EF1
:10643000588BD49AD48C12A101D0D58E12A301D03E
:10644000CD8012A501D0CA8412A701D0B18012AFAD
:1064500001D0F28E0BC5F8FF0CC5F7FF0DC5F6FF96
:106460000AC5E0FF09C5FAFF08C5FBFF02C5EAFF40
:1064700003C5E9FF04C5E2FF05C5E1FF06C5DAFF74
:1064800007C5D9FF01C5D8FF00C5E8FFE1009EAAF6
:1064900003D0AE509EBAFDD705EE19F00C0E166F64
:1064A000186BB1EC32F0EF6E59A105D0C0EC32F0B0
:1064B000185301E02CD0EF50EFEC32F0185303E00A
:1064C000598325D001D05993EF500D0A04E1000EF5
:1064D000EF6E4FD81CD0EF50080A0FE1190EE918E3
:1064E0000BE0080E12EC31F0200E12EC31F0080E29
:1064F00012EC31F0ED52162B08D0EE5012EC31F0C8
:10650000160703E1000EEF6E34D81653CAE11200ED
:10651000186B310A03E10A0E186F04D0030A02E176
:10652000140E186FB1EC32F0185310E00F0B18274F
:106530000A0E185F730EF76E480EF66E1851D8905B
:10654000F62601E3F72A0800F5CF18F5B1EC32F092
:106550001200E86A200E156FE806FEE11507FCE15F
:106560001200ABA202D0AB98AB889EAAFED7AE5069
:1065700012000D0E12EC31F00A0E12EC31F0120086
:106580002009136F680A02E1010E186F1351740A93
:1065900002E1020E186F13516C0A02E1030E186F2C
:1065A0001351640A02E1040E186F1351620A02E1EA
:1065B000050E186F1351770A02E1060E186F13517A
:1065C000720A02E1070E186F1351730A02E1080EF6
:1065D000186F13516D0A02E1090E186F12001B0AA1
:1065E0000AE1B1EC32F0EF6E5B0A05E1B1EC32F09A
:1065F000EF6E88EC32F01200185302E002EC33F038
:10660000196B1200FB6A660EFA6ED8901837D89094
:106610001837200ED890182501E3FA2A1851F926C8
:10662000000000002AEF33F031EF33F035EF33F0A4
:1066300040EF33F04BEF33F04EEF33F055EF33F0E4
:106640005BEF33F061EF33F064EF33F06BEF33F077
:1066500072EF33F0700EF76EC00EF66E0BEC31F089
:106660001200589D589BFF001200588D92D8A2D856
:106670005985280E146FA9EC32F01407FCE1FF00D5
:10668000D8EC36F0710EF76E140EF66E0BEC31F09E
:106690001FEC37F012000AEC35F01200720EF76EA4
:1066A000760EF66EB8DD64DA120080EC31F039B99E
:1066B00001D03981120080EC31F039B901D0398331
:1066C0001200E3EC37F01200730EF76EF60EF66E62
:1066D0000BEC31F01200730EF76EFE0EF66E0BEC43
:1066E00031F01200740EF76E060EF66E0BEC31F000
:1066F0007BEC33F0120047EC32F0050EEA6E190E17
:10670000E96E740EF76EBA0EF66E0BEC31F0000EF9
:10671000F86E23EC38F037C5F7FF000EF66EFF0E6B
:10672000156F100E166F100E161911E1F850B9EC16
:1067300037F0200E12EC31F0F750B9EC37F0F638A4
:1067400012EC38F012EC31F0200E12EC31F00900AE
:10675000F6A003D0F5CF14F506D0F550B9EC37F01C
:106760001451B9EC37F0F6B003D0200E12EC31F032
:106770001607000E161908E10D0E12EC31F00A0E84
:1067800012EC31F0100E166F1507CDE1B9EC32F0B6
:106790001200000EF86EF76EF66E21EE80F02AD928
:1067A000400EF626D8B0F72ADD52D952F8E1DA5277
:1067B000F6E11200396BBDEC30F0710EF76E9A0EF7
:1067C000F66E0BEC31F0B1EC32F03A0AD8A4FBD7FC
:1067D000326B17EC34F01F0B316FD890313317EC5C
:1067E00034F0336F17EC34F0346F17EC34F0356F4E
:1067F000010AD8B40BD03551020AD8B409D029EC1B
:1068000034F039BF13D039BD11D0DDD717EC34F0D7
:1068100080EC31F039B90AD0710EF76EDA0EF66EEF
:106820000BEC31F0B1EC32F0CBEC34F01200B1EC07
:1068300032F0BF0FD8A0070F0A0F376F373BB1EC0C
:1068400032F0BF0FD8A0070F0A0F37133751322786
:10685000120005EE19F031C516F517EC34F0EE6EA6
:1068600017EC34F0EE6E162FF8D717EC34F03253E5
:10687000D8B402D0398D15D03551040AD8B407D018
:106880003551D8A40ED075D839AF0FD80AD01A51C7
:10689000300AD8A406D0B1EC32F03A0AD8A4FBD71B
:1068A00000D02E0E12EC31F01200000EF86E33C53F
:1068B000F7FFF80E3415F66E050EEA6E290EE96E36
:1068C000040E166FF0EC34F0070E3415146F290E19
:1068D0001425E96E050EEA6E050EE26E190EE16EE4
:1068E000D890143331C516F5E6CFEEFFE6CFEEFFB4
:1068F000142B1607D8B404D01451040AD8A4F4D722
:10690000000EF86E33C5F7FFF80E3415F66E050E5F
:10691000EA6E290EE96EDDEC34F01653D8B4C1D717
:106920000900050EEA6E290EE96E16C514F5040E6F
:10693000166FF0EC34F014C516F5050EEA6E290E4C
:10694000E96EE6CFEEFFE6CFEEFF162FA1EF34F0B3
:10695000050EEA6E290EE96EF86A33C5F7FFF80EE8
:106960003415F66E080EF626D8B0F72ADDEC34F0B2
:10697000120033C55EF534C55FF531C560F5399F4A
:10698000600E335D07E605E1000E345D01E6398FE8
:1069900001D0398F1200740EF76E9A0EF66E0BEC62
:1069A00031F05E51B9EC37F0D8906035FE0F5F25BD
:1069B000B9EC37F0B9EC32F01200040E146F0A0093
:1069C000EECFF5FF0F00EECFF5FF0F00142FE0EF35
:1069D00034F0A68EA69CA68401EC35F0A694120095
:1069E0000900F5CFEEFF0900F5CFEEFF162FF0EF0F
:1069F00034F01200A68EA69CA684A68801EC35F081
:106A00001200D4AE06D0550EA76EAA0EA76EA682AF
:106A100000001200730EF76E920EF66E0BEC31F062
:106A2000730EF76E580EF66E0BEC31F047EC32F049
:106A300005EE19F059B348D0EF5244E0EE52EF5250
:106A40001EE1ED52EF502009720A0AE16EEC35F0BA
:106A5000730EF76E760EF66E0BEC31F03ED00ED064
:106A6000EF502009640A04E190EC35F036D006D0EE
:106A7000740EF76E6C0EF66E0BEC31F022D0ED5208
:106A8000040E156F5A8D5AAD03D0EE50BBEC36F0A4
:106A90001507F9E15AAD0FD0EF5206E179EC35F068
:106AA00090EC35F01AD006D0740EF76E6C0EF66EC0
:106AB0000BEC31F006D0740EF76E6C0EF66E0BEC2C
:106AC00031F001D00AD008D0B9EC32F0740EF76E74
:106AD0006C0EF66E0BEC31F0A3D71200588D588F68
:106AE000D4880F0EB912FF0EB86EFF0EB76ED49891
:106AF0001200588D589F05EE19F01FEEB8F0D4889B
:106B0000F00EB916020E156F23EC38F037C5E5FF0D
:106B1000EE501507F9E1D890B832B732D498120088
:106B2000D4880F0EB9140F0A1BE0730EF76E640EB3
:106B3000F66E0BEC31F0300E12EC31F0780E12ECF8
:106B400031F0D890B736B836B850B9EC37F0B75006
:106B5000B9EC37F0D890B832B732B9EC32F006D091
:106B6000730EF76E760EF66E0BEC31F0D4981200C1
:106B7000730EF76E040EF66E0BEC31F047EC32F04C
:106B800059B315D005EE19F0EF520FE024EC36F0B2
:106B90005ABF04D0E1EC35F013D006D0740EF76E76
:106BA0006C0EF66E0BEC31F001D00AD008D0B9ECC7
:106BB00032F0740EF76E6C0EF66E0BEC31F0D8D727
:106BC00012000A0E156F15EE3AF0E7AE07D05DC55C
:106BD000E6FF5CC5E6FF5BC5E7FF35D0E4505C1916
:106BE00025E1E4505B1921E15D531AE1E552E552DC
:106BF000E2CFEAFFE1CFE9FFEE52EE52EE52150787
:106C000002E1E78E0CD0EFBE07D0EECFE6FFEECF6D
:106C1000E6FFEECFE6FF02D0E78E01D0F0D704D03A
:106C2000E552E5525DC5E7FF0ED001D0E6521507EB
:106C300008E1740EF76E820EF66E0BEC31F003D0A5
:106C400001D0E652C2D712005A6B5B6B5C6B5D6B76
:106C500005EE19F0030E156F5A8D5B390F0B5C6F43
:106C60005B39F00B5B6FEF502CEC38F05B135AADD7
:106C700003D0EE50BBEC36F01507EFE15AAD07D06C
:106C8000060E5C5D04E65C510F0A01E05A9D5AADA8
:106C900054D0EF5201E150D0EF502009200A47E0D4
:106CA000EF502009610A09E1300E5D1504E1300E54
:106CB000300B5D1301D05A8F3AD0EF502009620A91
:106CC00012E1300E5D150DE15D510F0B08E15DBD68
:106CD00004D0300E200B5D1301D05A8F01D05A8F93
:106CE00001D05A8F24D0EF502009680A09E1300EF4
:106CF0005D1504E1300E100B5D1301D05A8F17D0D3
:106D0000EF5020092D0A0CE15DBD08D05D51300B1C
:106D1000200A02E05D8D01D05A8F01D05A8F07D032
:106D20005D510F0B03E1A7EC36F001D05A8F5AAF3B
:106D300001D002D0EC52ADE101D05A8F5ABF06D03B
:106D40005D510F0B03E15DAD01D05A8F1200EF5082
:106D5000200931080EE7090F0AE65D51300B200AC1
:106D600002E15A8F03D0EF500F0B5D1301D05A8F01
:106D700001D05A8F12005A9D2009146F2F080AE77C
:106D80000A0F02E65A8D06D01451600803E7060F79
:106D900001E65A8D1200050EE26E3A0EE16E0A0E01
:106DA000146F800EE66EE66AE66A1407FAE11200D6
:106DB000720EF76EE60EF66E0BEC31F001D8120093
:106DC00015EE3AF00A0E156FE7AE02D035D02ED090
:106DD000E7CF5DF5E45012EC38F012EC31F0E450FE
:106DE000B9EC37F05DAD02D02D0E01D0200E12ECC3
:106DF00031F05D51300B300A08E15D510F0BFB0F94
:106E000002E6020F01D0010E0FD05D51300B200AB7
:106E100002E1050E09D05D510F0BFD0F02E6010FD7
:106E200001D0000EE846010FDCEC37F0150702E157
:106E300003D001D0E652C8D7B9EC32F012000E519F
:106E400098D80F5196D8010EB7D8005192D8010E9C
:106E5000B3D801A502D0310E01D0300E12EC31F0C2
:106E6000200E12EC31F001A102D0310E01D0300E13
:106E700012EC31F0200E12EC31F001A902D0310EEB
:106E800001D0300E12EC31F0010E96D802516DD8BF
:106E900003516FD8020E90D8045167D8055169D8B4
:106EA000020E8AD8065161D8075163D8020E84D8E1
:106EB0005DEC37F0B9EC32F0120015EE3AF00A0E44
:106EC000156FE7AE02D02DD026D0E7CF5DF5E4CF29
:106ED000EAFFE4CFE9FF5D510F0B01E15D2B050EE9
:106EE000146F5DBD08D092EC37F0EE525D075D5136
:106EF0000F0BF9E10DD05D510F0BFF0FE92601E3F8
:106F0000EA2A92EC37F0ED525D075D510F0BF9E183
:106F10001451DCEC37F0150702E103D001D0E65242
:106F2000D0D712005D51300B300A0AE1EF50D0EC9F
:106F300037F012EC31F01451FF0F01E0140714D0B8
:106F40005D51300B200A06E1EF50C3EC37F0010E23
:106F5000146F0AD0EF50B9EC37F01451050A02E172
:106F6000030E01D0010E146F12005CD812EC31F048
:106F70001200136F133956D812EC31F0135152D856
:106F800012EC31F01200136F080E166F133702E384
:106F9000310E01D0300E12EC31F01607F7E112007D
:106FA000136F810F02E32A0E06D01351E00F02E2A5
:106FB0002A0E01D013511200136F200E12EC31F083
:106FC0001307FCE11200710EF76E180EF66E0BEC53
:106FD00031F047EC32F005EE19F0EF503DD8386F44
:106FE000EC5023EC38F037C536F5EC5003E1FDECFE
:106FF00037F002D019EC38F01200710EF76E760EF1
:10700000F66E0BEC31F038C5E2FF36C5E1FFE7382C
:1070100009D812EC31F0E75005D812EC31F0B9EC98
:1070200032F012000F0BF60F02E23A0F01D0410FBF
:10703000120038C5E2FF36C5E1FFEC5023EC38F012
:1070400037C5E7FF1200EF5007D8376F373BEC50DA
:1070500003D837133751120020099F0F02E30A0F9C
:1070600001D0310F1200FC060D0E12EC31F00A0EA9
:1070700012EC31F0FC50B9EC37F03A0E12EC31F072
:10708000FE50B9EC37F0FD50B9EC37F00D0E12ECB4
:1070900031F00A0E12EC31F0FC2A12000D0A090937
:1070A000095177696B42756720666F7220504943BA
:1070B0003138463435322076312E322E330D0A00E7
:1070C0000D0A463109463209463309463409463528
:1070D0000946360946370946380946390D0A4865D2
:1070E0006C70097265736554094C6F616409446979
:1070F00073706C617909427265616B0957617463E1
:10710000680952756E0953746570094D6F6469663C
:10711000790D0A0051423E00446973706C61792F09
:107120004D6F6469667920636F6E74656E74732049
:107130006F662052414D206F7220726567697374CB
:10714000657220616464726573733A200D0A3C6154
:1071500061613E20746F20446973706C6179202CEA
:107160003C6161612078783E20746F204D6F6469C6
:1071700066790D0A0000436F6E74656E7473202883
:10718000486578293A200000457261736520436F95
:107190006D706C6574652E2E2E00557365722070AF
:1071A000726F6772616D206D656D6F7279206572A7
:1071B00061736564202D2053656E64204845582016
:1071C00066696C65206E6F770D0A000052756E6EF1
:1071D000696E672E2E2E0D0A00000D0A446F776E21
:1071E0006C6F6164207375636365737366756C0D92
:1071F0000A000D0A5472616E736D697420457272D3
:107200006F72202D20436865636B73756D0D0A00E6
:107210000D0A57726974696E67206F7574736964BB
:1072200065205573657220416464726573732053E1
:10723000706163650D0A00000D0A4E6F207573655D
:107240007220636F64652072657365742076656370
:10725000746F72206973206C6F616465640D0A003D
:107260004E6F205573657220436F6465204C6F61CB
:107270006465640D0A00456E7465722077617463FD
:1072800068207661726961626C652E204578616D57
:10729000706C65733A207C20303132207C20303194
:1072A000322062207C2030313220612038207C2046
:1072B0003031322032207C203031322032202D20DB
:1072C0007C0D0A004D75737420626520616E20414B
:1072D00063636573732042616E6B206164647265E1
:1072E00073730D0A000020504320205720205A209D
:1072F00043204E20465352302046535231204653AD
:10730000523220002046363E000009095177696B51
:10731000427567204175746F7374617274696E672A
:10732000205573657220436F64650D0A00000909DA
:10733000507265737320616E79206B657920746F6C
:107340002061626F727420000001020304050006D0
:107350000708090A000B0C002046353E00002020DB
:1073600042503E0020202020427265616B706F69A0
:107370006E74203D2000202020204E6F2062726518
:10738000616B706F696E74206973207365740D0A88
:1073900000003C616161613E20746F207365742060
:1073A000627265616B706F696E742C2027522720A2
:1073B000746F2072656D6F766520627265616B70A7
:1073C0006F696E742C2027442720746F20646973C2
:1073D000706C617920627265616B706F696E740D9B
:1073E0000A00526573657420436F6D706C65746537
:1073F0002E200A0D0000463130200D0A00004631D3
:1074000031200D0A00004631323A456E7465722013
:107410004869676820416464726573732832206824
:10742000657820646967697473293E0042726F77DA
:107430006E2D6F7574205265736574204465746594
:10744000637465640A0D0000537461636B204F76AA
:107450006572666C6F770A0D0000537461636B2070
:10746000556E646572666C6F770A0D002046363E75
:10747000496E76616C696420436F6D6D616E640A5C
:107480000D002046363E5761746368204172726178
:10749000792046756C6C0A0D000048696768657351
:1074A0007420416464726573732050726F677261F7
:1074B0006D6D65643A203078000020202020202067
:1074C000203020312020322033202034203520204D
:1074D00036203720203820392020412042202043E8
:0A74E000204420204520460D0A003C
:020000040030CA
:0E000000FFFAFCFEFFFF7BFFFFFFFFFFFFFF8D
:00000001FF
